:200000003BC0CCC154C053C052C051C050C04FC04EC04DC04CC04BC04AC049C048C047C09B
:2000200046C045C044C0040309041C037700770077002E00660069007300630068006C0072
:200040002E00640065000E0355005300420061007300700012011001FF000008C016DC0588
:2000600002010102000109021200010100801909040000000000000011241FBECFE5D4E03A
:20008000DEBFCDBF10E0A0E6B0E0EEEDFFE002C005900D92A436B107D9F710E0A4E6B0E015
:2000A00001C01D92A73AB107E1F719D597C7A8CF85B7836085BF8BB780648BBF08950F938A
:2000C0001F93CF93DF9360918B00161604F5635080918800CBE9D0E0C81BD10980918700F4
:2000E0008D3209F44DC08091640087FD4EC0CE010DD58F3F09F485C0882309F05AC02FEF93
:2001000030E0309364002093600010928B008091610084FF29C0809160008F3F29F1682F9A
:20012000893008F03DC0861B809360008091640080FF34C003EC8F5F8093640087FD69C014
:20014000662309F455C08CE790E0A6D5682F7727162F693008F479C08FEF809360009EE1EE
:2001600000937B00909361009AE086B3837009F0F7C09150D1F710928C0010928600F0C0E8
:200180008AE5809361006830B9F020E030E8309364002093600010928B00B9CF0BE4CBCFAB
:2001A00068E0861B809360008091640080FFF6CFC1CF20E030E0EBCF8881807609F05CC0BC
:2001C00024E830E0109284008981882309F05BC01092850030938A002093890022E030E84A
:2001E0008F818823A1F68E81821788F6282FCFCF60E08CE790E0CED094E08FEF809360006C
:20020000AFCF809360008EE1809361002FEF30E078CF2091890030918A0086FD1FC0462F39
:2002200041504F3F61F0F901942FACE7B0E081918D939150E0F7240F311D2F5F3F4F309324
:200240008A0020938900772783CF8CE790E0A2D0912F9C5F183008F083CFCFCF462F4150A2
:200260004F3F69F3F901942FACE7B0E084918D9331969150D8F7DFCFCE0160D5282F8F3F31
:20028000A9F030E8ADCF853059F08630A9F08830E9F0893021F18A3041F120E030E8A0CF15
:2002A0008A8180938C0020E030E89ACF888187FF27CF2E8130E025CF8B818130E9F0823093
:2002C00081F1833011F120E030EC8ACF8EE890E090938A008093890021E030E881CF8A81DF
:2002E00080938E0020E030E87BCF30938A002093890021E030E874CF84E590E090938A0090
:200300008093890022E130EC6BCF8A81882391F486E290E090938A008093890024E030EC6C
:200320005FCF86E690E090938A008093890022E130EC56CF813059F0823029F686E490E081
:2003400090938A00809389002EE030EC49CF8AE290E090938A00809389002CE130EC40CFB5
:20036000DF91CF911F910F910895A82FB92F80E090E041E050EA60956F5F58F42D9138EFE2
:2003800082279795879510F0842795273F5FC8F3F3CF0895EADF8D939D930895CF93CFB7AF
:2003A000CF93B09BFECFB09B09C0B09B07C0B09B05C0B09B03C0B09B01C0A1C0DF93C0914F
:2003C0008800DD27C157DF4FB09B02C0DF91EBCF2F930F931F9306B32FEF00FB20F94F9331
:2003E0003F9316B34FEF012700FB21F93BE031C04E7F012F16B3216028C0102F4D7F22601F
:20040000000006B329C04B7F2460012F000016B32BC016B3477F28602AC04F7E06B3206100
:200420002CC04F7D16B320622FC04F7B06B3206432C0422706B349934FEF0000102710FB53
:2004400020F916B31370C9F1297F91F2012700FB21F906B3237F89F2315058F1102710FB33
:2004600022F916B3277E79F2012700FB23F92F7C81F206B3102710FB24F92F7971F200C048
:2004800016B3012700FB25F92F7359F200C006B3102710FB26F9223040F200C016B3012756
:2004A00000FB27F9243028F64F77206816B30000F9CF10E41ABF002717C03B503195C31BD6
:2004C000D04010E41ABF0881033CE9F00B34D9F0209186001981110F1213EDCF093641F153
:2004E0000D3211F0013E39F700938D003F914F911F910F912F91DF91CAB7C6FD52CFCF9138
:20050000CFBFCF91189500918D00002379F310918B00112349F534304AF130938B00009375
:200520008700109188003BE0311B309388001EC000918B000130C4F40AE53091610034FD34
:2005400017C000936100CBE7D0E016C0052710E008BB1FC0052722C0052727C005272CC0A1
:20056000052710E008BB33C04AE503C042ED01C0432FC4E1D0E032E017B31360C09A08B39C
:2005800017BB5F9353E020E820FF052708BB279517951C3FD8F620FF0527279508BB179547
:2005A0001C3FC0F620FF05272795179508BB1C3F98F620FF0527279517951C3F08BB70F694
:2005C00000C0499120FF052708BB279517951C3F38F620FF0527279508BB17951C3F38F584
:2005E00020FF05272795179508BB1C3F10F520FF0527279517951C3F08BBE8F4242F3A9556
:2006000019F60C7F5F9108BB10918C00110FC651D04011F01093860010E41ABF016017B3F7
:200620001C7F402F4C7F08BB17BB48BB5FCF0527D3CF0527D8CF0527DDCF8091620084307F
:2006400041F0853051F0833069F083E58DB91EB8089581E58DB91EB8089581E58DB981E01A
:200660008EB9089582E58DB981E08EB9089580916200813039F085E793E09093A60080939C
:20068000A50008951DB888E593E09093A6008093A500089592B782B7891B8C30E0F30895F3
:2006A00087B3837D87BB88B3837D88BB1DB80895FF920F931F93182FFF2400E00CC0C39878
:2006C000FF0CB499F394C59AE5DFC598E3DF0F5F083029F0110F17FFF2CFC39AF1CF8F2D6A
:2006E00099271F910F91FF9008958FB9779BFECF8FB1992708950F931F930FE11DC0E09168
:20070000A500F091A6000995182FE091A500F091A60080E00995133569F11DB8C59ABADF7E
:20072000C598B8DF8091A5009091A6008557934021F101500F3F21F1E091A500F091A60099
:200740008CEA0995E091A500F091A60083E5099580916500882399F2E091A500F091A60059
:2007600080E00995E091A500F091A60080E00995893699F680E090E005C05FDF0150E0F6F8
:2007800081E090E01F910F910895EF92FF920F931F937B018C0180916500882321F58E2D3A
:2007A0008170880F880F880FE091A500F091A60080620995D801C70129E0B695A795979569
:2007C00087952A95D1F7E091A500F091A600099516950795F794E794E091A500F091A60011
:2007E0008E2D099515C0E091A500F091A60080E20995BB27A12F902F8F2DE091A500F091CA
:20080000A6000995E091A500F091A6008E2D0995E091A500F091A60080E0099599271F9153
:200820000F91FF90EF900895CF93DF93EC01809165008130D9F0E091A500F091A60080EA15
:2008400009958D2F9927E091A500F091A6000995E091A500F091A6008C2F0995E091A500F7
:20086000F091A60080E00995992702C080E090E0DF91CF9108951F93CF93DF93EC01162FDC
:20088000809165008130D9F0E091A500F091A60080EC09958D2F9927E091A500F091A60068
:2008A0000995E091A500F091A6008C2F0995E091A500F091A600812F09958EE103D180E0D6
:2008C00090E0DF91CF911F910895CF92DF92EF92FF920F931F937B018C01D42E80916500D2
:2008E0008130D9F1E091A500F091A6008CE40995D801C70179E0B695A795979587957A955A
:20090000D1F7E091A500F091A6000995D801C701B695A79597958795E091A500F091A60087
:200920000995E091A500F091A60080E009958FEFD816B1F0C2B65EE1D52EC801B70125DF92
:200940008F3F59F482B78C198D3310F0C2B6DA94DD2099F781E090E007C080E090E004C03F
:200960008FE0B0D080E090E01F910F91FF90EF90DF90CF900895CF92DF92EF92FF920F9369
:200980001F937B018C01D42EC22E80916500813009F442C08E2D8170880F880F880FE091A2
:2009A000A500F091A60080640995D801C70129E0B695A795979587952A95D1F7E091A500D3
:2009C000F091A6000995D801C701B695A79597958795E091A500F091A6000995E091A500F1
:2009E000F091A6008D2D0995CC20B1F18FE7D816B1F1C2B6EEE1DE2EC801B701C6DE8F37A6
:200A000059F582B78C198D3310F0C2B6DA94DD2099F781E090E027C0E091A500F091A60082
:200A200080E40995BB27A12F902F8F2DE091A500F091A6000995E091A500F091A6008E2DB4
:200A40000995E091A500F091A6008D2D099592B782B7891B8435E0F380E090E004C08FE0AE
:200A600031D080E090E01F910F91FF90EF90DF90CF90089587B38C6287BB80916500882351
:200A800081F4C298C5988EE11DD0C29A8EE11AD0C2988091A5009091A6008557934081F022
:200AA0000895C29AC5988EE10DD0C2988EE10AD0C29A8091A5009091A6008557934081F7F1
:200AC000BCDD0895382F882349F020E092B782B7891B8C33E0F32F5F3217C1F7089512BAE5
:200AE00018BA8BEF81BB8FEF87BB9EEF9150F1F78150E1F717BA93E094BB8EEF85BB93BF0D
:200B0000B6DDD6DA7894DBDADADAFDCFBF92CF92DF92EF92FF920F931F93CF93DF937C0177
:200B2000C62E80916600813029F0843019F08FEF90E0A8C0CC2009F4A3C0BB24DD245AC027
:200B40008091760090917700892B09F065C0CD2DDD27F701EC0FFD1F6091720070917300C0
:200B6000809174009091750021E0408104DF80916700909168000197909368008093670017
:200B8000892BF9F4109266008091780081FF41C02091790030917A0080917600909177001E
:200BA00028173907B1F1CE0DDF1D60917200709173008091740090917500488186DE91E0AD
:200BC000B92E8091720090917300A0917400B09175000196A11DB11D80937200909373007E
:200BE000A0937400B0937500D394CD1409F445C080916600813009F4A3CFCD2DDD27F701BF
:200C0000EC0FFD1F6081809172009091730033DEAECF81E0B82ED5CFCD2DDD2787010C0FAB
:200C20001D1F6091720070917300809174009091750020E0F80140819EDE809179009091A5
:200C40007A00019790937A0080937900892B09F08ECF6091720070917300809174009091D2
:200C60007500F801408131DE809176009091770090937A00809379007ACF8B2D992702C06B
:200C800080E090E0DF91CF911F910F91FF90EF90DF90CF90BF9008950F931F93CF93DF9374
:200CA000EC01062F90916600892F8250823018F08FEF90E03EC06623C1F110E021C080913E
:200CC000720090917300B0DDFE01E10FF11D80838091720090917300A0917400B09175000F
:200CE0000196A11DB11D8093720090937300A0937400B09375001F5F011791F090916600B9
:200D00009230E9F6609172007091730080917400909175003ADDFE01E10FF11D8083D8CF82
:200D2000083018F0802F992704C010926600802F9927DF91CF911F910F910895CF93DF9338
:200D4000EC018981813009F485C0823009F4BAC0833009F4BCC0843001F1873009F488C0B2
:200D6000853009F426C1863009F441C0883009F4D1C0893079F481E0809369008A819B81B6
:200D8000AC81BD818093720090937300A0937400B093750020E030E017C180916900882361
:200DA000A1F48B812A819927982F88273327822B932BAA2797FDA095BA2F809372009093C1
:200DC0007300A0937400B09375008F812E819927982F88273327822B932B909368008093E9
:200DE000670082E0809366002FEF30E0EDC080916900882309F4B3C08C819D819F709093E4
:200E000078002D813327207F307022953295307F3227207F3227280F311D30937700209323
:200E2000760080916500813009F4C9C090FD8EC08F812E819927982F88273327822B932BFA
:200E4000909368008093670081E0809366002FEF30E0BAC08A81809362008B818093650007
:200E600006DC1092690006DEA99820E030E0ACC0809169008823A1F48B812A819927982FEC
:200E800088273327822B932BAA2797FDA095BA2F8093720090937300A0937400B0937500E1
:200EA0008F812E819927982F88273327822B932B909368008093670083E0809366002FEF79
:200EC00030E082C0EDDBA99A20E030E07DC0E091A500F091A6008A81099580936A00E09194
:200EE000A500F091A6008B81099580936B00E091A500F091A6008C81099580936C00E09126
:200F0000A500F091A6008D81099580936D0024E030E05AC0809169008823B1F110927700CB
:200F200010927600109278008F812E819927982F88273327822B932B9093680080936700C0
:200F400084E0809366002FEF30E03EC0809176009091770090937A008093790069CF8B81FC
:200F60002A819927982F88273327822B932BAA2797FDA095BA2F8093720090937300A093FA
:200F80007400B093750038CF8B812A819927982F88273327822B932BAA2797FDA095BA2FE9
:200FA0008093720090937300A0937400B0937500B5CFA1DB80936A0021E030E005C01092C2
:200FC00077001092760032CF8AE690E090938A0080938900C901DF91CF910895FFCFFF5AFA
:020FE00001000E
:00000001FF
